:107800000C94343C0C94513C0C94513C0C94513CE1
:107810000C94513C0C94513C0C94513C0C94513CB4
:107820000C94513C0C94513C0C94513C0C94513CA4
:107830000C94513C0C94513C0C94513C0C94513C94
:107840000C94513C0C94513C0C94513C0C94513C84
:107850000C94513C0C94513C0C94513C0C94513C74
:107860000C94513C0C94513C11241FBECFEFD8E036
:10787000DEBFCDBF11E0A0E0B1E0E4EAFFE702C067
:1078800005900D92A230B107D9F712E0A2E0B1E065
:1078900001C01D92AD30B107E1F70E942D3D0C945F
:1078A000D03F0C94003C982F95959595959595957E
:1078B000905D8F708A307CF0282F295A8091C0000B
:1078C00085FFFCCF9093C6008091C00085FFFCCF60
:1078D0002093C6000895282F205DF0CF982F809127
:1078E000C00085FFFCCF9093C6000895EF92FF92F1
:1078F0000F931F93EE24FF2487018091C00087FD22
:1079000017C00894E11CF11C011D111D81E2E8164D
:1079100081EAF80687E0080780E0180770F3E09135
:107920000401F091050109958091C00087FFE9CF1E
:107930008091C6001F910F91FF90EF9008950E94D3
:10794000763C982F8091C00085FFFCCF9093C600B5
:1079500091362CF490330CF09053892F089597555D
:10796000892F08951F930E949F3C182F0E949F3CCF
:107970001295107F810F1F9108951F93182F882350
:1079800021F00E94763C1150E1F71F9108951F935A
:10799000182F0E94763C803249F0809103018F5F5E
:1079A000809303018530C1F01F9108958091C0003C
:1079B00085FFFCCF84E18093C6008091C00085FFE5
:1079C000FCCF1093C6008091C00085FFFCCF80E102
:1079D0008093C6001F910895E0910401F091050184
:1079E00009951F9108950E94763C803241F0809164
:1079F00003018F5F80930301853081F008958091AA
:107A0000C00085FFFCCF84E18093C6008091C00058
:107A100085FFFCCF80E18093C6000895E0910401CA
:107A2000F09105010995089548EC50E08823A1F0F4
:107A30002D9A28EE33E0FA013197F1F721503040CA
:107A4000D1F72D9828EE33E0FA013197F1F7215064
:107A50003040D1F7815061F708953F924F925F9285
:107A60006F927F928F929F92AF92BF92CF92DF924E
:107A7000EF92FF920F931F93CF93DF939FB7F894EA
:107A800080E88093610081E0809361000000000045
:107A9000000000009FBF000082E08093C00080E1F2
:107AA0008093C4001092C50088E18093C10086E0F5
:107AB0008093C2005098589A259A81E00E94143D04
:107AC00024E1F22E9EE1E92E85E9D82E0FE0C02EAA
:107AD00010E1B12EAA24A394B1E49B2EA6E58A2E30
:107AE000F2E57F2EE0E26E2E79E4572E63E5462E16
:107AF00050E5352E0E94763C8033B1F18133B9F1E7
:107B0000803409F46FC0813409F476C0823409F4FA
:107B100085C0853409F488C0803531F1823521F182
:107B2000813511F1853509F485C0863509F48DC09C
:107B3000843609F496C0843709F403C1853709F403
:107B400072C1863709F466C0809103018F5F80930C
:107B50000301853079F6E0910401F0910501099562
:107B60000E94763C803351F60E94F33CC3CF0E94C2
:107B7000763C803249F78091C00085FFFCCFF092BF
:107B8000C6008091C00085FFFCCF9092C600809116
:107B9000C00085FFFCCF8092C6008091C00085FFA9
:107BA000FCCF7092C6008091C00085FFFCCF609230
:107BB000C6008091C00085FFFCCF5092C600809126
:107BC000C00085FFFCCF4092C6008091C00085FFB9
:107BD000FCCF3092C6008091C00085FFFCCFB092F0
:107BE000C60088CF0E94763C863808F4BDCF0E943C
:107BF000763C0E94F33C7ECF0E94763C803809F4AC
:107C00009CC0813809F40BC1823809F430C188392D
:107C100009F48FC080E00E94C73C6CCF84E10E94D1
:107C2000BD3C0E94F33C66CF85E00E94BD3C0E94B3
:107C3000F33C60CF0E94763C809306010E94763C24
:107C4000809307010E94F33C55CF0E94763C80331D
:107C500009F411C183E00E94BD3C80E00E94C73C52
:107C600049CF0E94763C809309020E94763C809323
:107C7000080280910C028E7F80930C020E94763C59
:107C8000853409F409C18091080290910902892B79
:107C900089F000E010E00E94763CF801E85FFE4FBA
:107CA00080830F5F1F4F809108029091090208178F
:107CB000190788F30E94763C803209F045CF809105
:107CC0000C0280FFF5C06091060170910701660FFC
:107CD000771F7093070160930601A0910802B0918D
:107CE00009021097C9F0E8E0F1E09B01AD014E0FE9
:107CF0005F1FF999FECF32BD21BD819180BDFA9AF7
:107D0000F99A2F5F3F4FE417F50799F76A0F7B1F2A
:107D100070930701609306018091C00085FFFCCF3E
:107D2000F092C6008091C00085FFFCCFB092C600E3
:107D3000E1CE83E00E94C73CDDCE82E00E94C73CDA
:107D4000D9CE0E94763C809309020E94763C8093B3
:107D500008028091060190910701880F991F909366
:107D60000701809306010E94763C853409F49AC08D
:107D700080910C028E7F80930C020E94763C8032B0
:107D800009F0B8CE8091C00085FFFCCFF092C6000C
:107D9000A0910802B09109021097C1F180910C02E4
:107DA000082F0170182F16951170E0910601F091BF
:107DB0000701AF014F5F5F4FBA0120E030E00023C1
:107DC000B1F4112339F494918091C00085FFFCCF68
:107DD0009093C6002F5F3F4FCB010196FA012A17FF
:107DE0003B0780F4BC014F5F5F4F002351F3F999CB
:107DF000FECFF2BDE1BDF89A90B58091C00085FF3D
:107E0000FCCFE6CF70930701609306018091C0001C
:107E100085FDE5CE8091C00085FFF8CFE0CE81E002
:107E20000E94C73C67CE0E94763C803209F08CCE1F
:107E30008091C00085FFFCCFF092C6008091C00009
:107E400085FFFCCFE092C6008091C00085FFFCCF8B
:107E5000D092C6008091C00085FFFCCFC092C600C2
:107E60008091C00085FFFCCFB092C60043CE80E178
:107E70000E94C73C3FCE0E94763C0E94763C182F61
:107E80000E94763C112309F483C0113009F484C0A8
:107E90008FE00E94C73C2ECE80910C0281608093BF
:107EA0000C02F1CE80910C02816080930C0265CFB0
:107EB000809107018823880F880B8A2180930B0209
:107EC0008091060190910701880F991F90930701F7
:107ED000809306018091080280FF09C0809108020A
:107EE0009091090201969093090280930802F894F8
:107EF000F999FECF1127E0910601F0910701C8E042
:107F0000D1E08091080290910902103091F4009123
:107F1000570001700130D9F303E000935700E89552
:107F20000091570001700130D9F301E1009357002F
:107F3000E895099019900091570001700130D9F32C
:107F400001E000935700E8951395103498F011273D
:107F50000091570001700130D9F305E000935700FC
:107F6000E8950091570001700130D9F301E10093C9
:107F70005700E8953296029709F0C7CF103011F0FC
:107F80000296E5CF11248091C00085FFC5CEC8CEF2
:107F90008EE10E94C73CAECD85E90E94C73CAACDC8
:047FA000F894FFCF83
:027FA40080005B
:040000030000780081
:00000001FF
